:100000000C9437010C9454010C9454010C94540139
:100010000C9454010C9454010C9454010C9454010C
:100020000C9454010C9454010C9454010C945401FC
:100030000C9433130C9454010C9454010C945401FB
:100040000C9454010C94FA050C94561B0C94411218
:100050000C94D1120C9454010C9454010C9454013E
:100060000C9454010C9454010C9454010C945401BC
:100070004570692D4F5344205665722E302E392E0F
:10008000352E320000416B7475656C6C65732053BE
:10009000657474696E67000053657474696E6720D7
:1000A000200000486F6568656E73656E736F72201F
:1000B00000004853206D697420536368616C746557
:1000C0007220000048656164696E6720486F6C6447
:1000D0002000004B6F6D706173732000004B6F6DDB
:1000E0007061737320666978200000475053204187
:1000F0006B74697620000041636873656E6B6F7086
:1001000070656C756E67200000447265687261747A
:100110006520626567722E2000004665686C657216
:100120002046433C2D3E4F5344200000556E7465DD
:10013000727370616E6E756E672000004B65696E3C
:10014000652053657474696E672D416E7A656967C1
:1001500065000050432F425420616B7469760000A3
:1001600055656265726E65686D65204C65747A745C
:1001700065732053657474696E6700004B65696E22
:1001800065204465766976652D416E7A6569676597
:10019000000050432F425420616B74697600005573
:1001A000656265726E65686D65204C65747A74650C
:1001B000732044657669636500004F4E00002D2D65
:1001C0002D000044657669636520756E6420566570
:1001D0007273696F6E736162667261676500004475
:1001E000656369766520202020203D200000465769
:1001F0002D56657273696F6E203D200000464300E6
:10020000004E43000046432D6F6C642046570000AB
:100210004550492D4D656E750050616C0050432F5F
:100220004254004B656E6E756E670052432D4265F9
:100230007472696562004550492D5374726F6D0088
:1002400045786974004F4E002D2D0076767D7676C8
:100250007A76767E76767776767B76767876767C24
:1002600076767976767D76767A76767E7600112445
:100270001FBECFEFD4E0DEBFCDBF11E0A0E0B1E004
:10028000E4E3F9E302C005900D92A03BB107D9F772
:1002900014E0A0EBB1E001C01D92A231B107E1F77B
:1002A0000E9464010C94981C0C94000086E981BBA8
:1002B0008FE084BBAC9AAD9A8EE28ABB80EB87BBA1
:1002C000C69AD99ADD9A08951092F8011092F40115
:1002D0001092F901E199FECF80E090E09FBB8EBBC8
:1002E000E09A8DB38093B701E199FECF81E090E071
:1002F0009FBB8EBBE09A8DB380930801E199FECF3E
:1003000082E090E09FBB8EBBE09A8DB38093B801F2
:10031000E199FECF87E190E09FBB8EBBE09A8DB361
:100320008093C501E199FECF88E190E09FBB8EBB31
:10033000E09A8DB38093DE01E199FECF8AE190E0EF
:100340009FBB8EBBE09A8DB380931101E199FECFE4
:1003500089E190E09FBB8EBBE09A8DB38093DA0178
:10036000E199FECF8BE190E09FBB8EBBE09A8DB30D
:100370008093B90120910801213079F49EE0909397
:100380000B0187E080930C0186E880930D01209398
:100390000E0190930F018CE00EC09CE090930B0136
:1003A00085E080930C018AE480930D0110920E0188
:1003B00090930F018AE0809310010E9450180E94D0
:1003C00056010E94F3058091B701813019F40E9413
:1003D0001C1102C00E940C117894A89A0E941F055B
:1003E0000E945A060E944D0A8091B901882311F09B
:1003F0000E948D0A8091E301882311F00E9443142A
:100400000E948D0A8091B901813011F40E94A61BCF
:100410000E94ED118091D601813021F41092D60115
:100420000E94E8188091FD01813021F41092FD01B5
:100430000E94230E8091B2018130F1F41092B2013A
:100440008091F801882391F48091DA01843071F46D
:100450008091B701882351F480E091E066E00E942A
:100460002E1280E364E641E00E949B110E94261355
:100470000E942B130E9493158091B901813031F4B1
:100480008091FE01813011F40E94B11B8091B50171
:100490008130E1F48091F8018823C1F4AA9A0E9486
:1004A000470F0E94AD090E94C2088091E101882394
:1004B00021F00E949F130E940B0B8091E201882380
:1004C00011F00E9498180E94E20AAA988091B00147
:1004D000813009F03FC08091F8018823D9F510924E
:1004E000B0018091DA01823029F483E66FE64AE0B8
:1004F0000E949B118091DA01813029F482E664E642
:100500004AE00E949B118091C501882321F08091CF
:100510000A01833014F00E94BC0A8091C2019091BC
:10052000C30101969093C3018093C2010197CB97B9
:1005300069F48091C0019091C10101969093C1012D
:100540008093C0011092C3011092C2010E949B0CC3
:100550000E94E50D8091B101813009F05BCF80915F
:10056000F801882309F056CF1092B1018091B901AA
:10057000813039F48091FE01882319F481E00E94D2
:10058000B11B0E94560A8091E301882309F442CFEF
:100590000E949F140E941F140E940A150E9470144A
:1005A0000E944B140E94011435CF782FD99827E070
:1005B00030E041E050E0DB98000000000000000067
:1005C000CA01022E02C0880F991F0A94E2F78723FE
:1005D00011F0DA9A01C0DA98000000000000000073
:1005E000DB9A0000000000000000215030408FEF37
:1005F0002F3F380701F727E030E041E050E0DB987B
:100600000000000000000000CA01022E02C0880F96
:10061000991F0A94E2F7862311F0DA9A01C0DA985A
:100620000000000000000000DB9A00000000000055
:100630000000215030408FEF2F3F380701F7DB9843
:10064000DA98D99A089584E064E00E94D50280E0A7
:100650006CE40E94D5021092B2018091B20188230D
:10066000E1F38CE66AE00E94D50285E060E00E943A
:10067000D50208950F931F938091B0018823E1F371
:100680001092B0018091DA01823051F40E942C1155
:100690001092B0018091B0018823E1F31092B00173
:1006A0001092E0010E94470F82E661E74FEF0E943F
:1006B0009B1110E000E01DC08091B501813071F404
:1006C00080919902813519F40E94470F02C08091F0
:1006D000B50182E661E74FEF0E949B118091B00166
:1006E000813039F410E0023009F411E01092B001C9
:1006F0000F5F8091E001882311F41123E9F28091CA
:10070000DA01823011F40E947311112309F0D9C06B
:1007100080910104809311018091EB038093DE01AD
:100720002091DE01E199FECF88E190E09FBB8EBB76
:100730002DBB0FB6F894E29AE19A0FBE20911101F9
:10074000E199FECF8AE190E09FBB8EBB2DBB0FB637
:10075000F894E29AE19A0FBE82E061E045E850E049
:100760000E949F0E82E062E048E950E00E949F0EE6
:1007700082E064E043EA50E00E949F0E82E065E080
:1007800042EB50E00E949F0E82E066E044EC50E0B5
:100790000E949F0E82E067E043ED50E00E949F0EB2
:1007A00082E068E04DED50E00E949F0E82E069E03B
:1007B0004BEE50E00E949F0E82E06AE047EF50E06F
:1007C0000E949F0E82E06BE04CE251E00E949F0E7F
:1007D0004091DC015091DD0184E162E00E94F80D5E
:1007E0008091DE0180FF05C084E164E04AEB51E0C6
:1007F00004C084E164E04EEB51E00E949F0E8091C2
:10080000DE0181FF05C084E165E04AEB51E004C0F0
:1008100084E165E04EEB51E00E949F0E8091DE0185
:1008200082FF05C084E166E04AEB51E004C084E148
:1008300066E04EEB51E00E949F0E8091DE0183FF47
:1008400005C084E167E04AEB51E004C084E167E061
:100850004EEB51E00E949F0E8091DE0184FF05C0A7
:1008600084E168E04AEB51E004C084E168E04EEBCB
:1008700051E00E949F0E8091DE0185FF05C084E15A
:1008800069E04AEB51E004C084E169E04EEB51E0DD
:100890000E949F0E8091DE0186FF05C084E16AE020
:1008A0004AEB51E004C084E16AE04EEB51E00E9463
:1008B0009F0E4091110184E16BE050E00E94F80D21
:1008C00020C082E062E045E850E00E949F0E82E096
:1008D00065E04AE151E00E949F0EE199FECF88E178
:1008E00090E09FBB8EBBE09A8DB38093E703E199C4
:1008F000FECF8AE190E09FBB8EBBE09A8DB38093E0
:1009000011019091E703892F81708093E101892F74
:1009100088708093E201892F80728093E301947044
:100920009093E4011F910F9108951F938091B0015E
:100930008823E1F31092B0018091B0018823E1F3A4
:100940001092B00183E666E740E00E949B1110E040
:100950000DC08091B501813011F40E94E5108091A5
:10096000B001813019F41092B00111E08091DB01E7
:10097000882311F4112369F3112309F054C082E094
:1009800062E043EC51E00E949F0E82E064E04FED94
:1009900051E00E949F0E82E066E04EEE51E00E9420
:1009A0009F0E8091DA01813031F48EE064E04DEFEA
:1009B00051E00E949F0E8091DA01823031F48EE086
:1009C00064E041E052E00E949F0E8091DA018430A1
:1009D00031F48EE064E045E052E00E949F0E4091C9
:1009E000A1038EE066E050E00E94F80D4091A20362
:1009F00080E166E050E00E94F80D4091A30383E19E
:100A000066E050E00E94F80D2091DA01E199FECFF6
:100A100089E190E09FBB8EBB2DBB0FB6F894E29AA4
:100A2000E19A0FBE0AC0E199FECF89E190E09FBB39
:100A30008EBBE09A8DB38093DA011F9108950E94D6
:100A4000230383E66FE644E60E949B1180E06CE49A
:100A50000E94D5021092B0018091B0018823E1F389
:100A600087E062E040E750E00E949F0E0E945B0634
:100A70001092B0018091B0018823E1F31092B0018F
:100A80008091B0018823E1F31092B0018091B00110
:100A90008823E1F31092B0018091B0018823E1F343
:100AA0001092B00184E064E00E94D50280E06CE422
:100AB0000E94D5028091B701882319F40E94950401
:100AC0001CC082E062E04CE751E00E949F0E82E091
:100AD00064E042E951E00E949F0E82E066E04FE947
:100AE00051E00E949F0EE199FECF89E190E09FBB0B
:100AF0008EBBE09A8DB38093DA018091B001882398
:100B0000E1F31092B0018091B0018823E1F31092DB
:100B1000B00184E064E00E94D50280E06CE40E94B1
:100B2000D5028091B701882319F40E943A0326C0A8
:100B300082E062E04CE351E00E949F0E82E064E0BC
:100B400043E551E00E949F0E82E066E040E651E0FE
:100B50000E949F0EE199FECF88E190E09FBB8EBB83
:100B6000E09A8DB38093DE01E199FECF8AE190E0B7
:100B70009FBB8EBBE09A8DB3809311018091DA0107
:100B8000823029F483E66FE64AE00E949B1180914F
:100B9000DA01813029F482E664E64AE00E949B1182
:100BA0008091B0018823E1F31092B0018091B001EF
:100BB0008823E1F31092B0018091B0018823E1F322
:100BC0001092B0018091B0018823E1F31092B0013E
:100BD0008091B0018823E1F31092B00184E064E0D9
:100BE0000E94D502089582E083BF82E48EBD8AE030
:100BF00089BF08951F920F920FB60F9211248F9301
:100C00009F938091B4018F5F8093B4018091B40170
:100C1000883449F591E09093B3011092B40180912A
:100C200008048F5F8093080480910804843631F4AF
:100C3000109208049093B0019093B1018091080440
:100C4000823319F481E08093B101809107048F5FB2
:100C500080930704809107048A3029F410920704D6
:100C600081E08093B2019F918F910F900FBE0F9002
:100C70001F901895982F80538A3010F020E005C0FF
:100C8000903311F42AE001C0282F892F81548A3132
:100C900010F4292F2653892F81568A3110F4292FD9
:100CA0002C539D3211F429E403C09E3209F421E44F
:100CB000822F0895089585E060E00E94D50286E0C5
:100CC00063E80E94D50287E060E90E94D50285E0D2
:100CD00060E00E94D50286E064E80E94D50287E0C9
:100CE00061E90E94D50285E060E00E94D50286E0BD
:100CF00065E80E94D50287E062E90E94D50285E09E
:100D000060E00E94D50286E066E80E94D50287E096
:100D100063E90E94D50285E060E00E94D50286E08A
:100D200067E80E94D50287E064E90E94D50285E069
:100D300060E00E94D50286E068E80E94D50287E064
:100D400065E90E94D50285E060E00E94D50286E058
:100D500069E80E94D50287E066E90E94D50285E035
:100D600060E00E94D50286E06AE80E94D50287E032
:100D700067E90E94D50285E060E00E94D50286E026
:100D800061EA0E94D50287E068E90E94D50285E009
:100D900060E00E94D50286E062EA0E94D50287E008
:100DA00069E90E94D50285E060E00E94D50286E0F4
:100DB00063EA0E94D50287E06AE90E94D50285E0D5
:100DC00060E00E94D50286E064EA0E94D50287E0D6
:100DD0006BE90E94D50285E060E00E94D50286E0C2
:100DE00065EA0E94D50287E06CE90E94D50285E0A1
:100DF00060E00E94D50286E066EA0E94D50287E0A4
:100E00006DE90E94D50285E060E00E94D50286E08F
:100E100067EA0E94D50287E06EE90E94D50285E06C
:100E200060E00E94D50286E068EA0E94D50287E071
:100E30006FE90E94D50285E060E00E94D50286E05D
:100E40006FEB0E94D50287E060EA0E94D50285E040
:100E500060E00E94D50286E060EC0E94D50287E047
:100E600061EA0E94D50285E060E00E94D50286E03A
:100E700061EC0E94D50287E062EA0E94D50285E01B
:100E800060E00E94D50286E062EC0E94D50287E015
:100E900063EA0E94D50285E060E00E94D50286E008
:100EA00063EC0E94D50287E064EA0E94D50285E0E7
:100EB00060E00E94D50286E064EC0E94D50287E0E3
:100EC00065EA0E94D50285E060E00E94D50286E0D6
:100ED00065EC0E94D50287E066EA0E94D50285E0B3
:100EE00060E00E94D50286E066EC0E94D50287E0B1
:100EF00067EA0E94D50285E060E00E94D50286E0A4
:100F00006DED0E94D50287E068EA0E94D50285E077
:100F100060E00E94D50286E06EED0E94D50287E077
:100F200069EA0E94D50285E060E00E94D50286E071
:100F30006FED0E94D50287E06AEA0E94D50285E043
:100F400060E00E94D50286E060EE0E94D50287E054
:100F50006BEA0E94D50285E060E00E94D50286E03F
:100F600061EE0E94D50287E06CEA0E94D50285E01E
:100F700060E00E94D50286E062EE0E94D50287E022
:100F80006DEA0E94D50285E060E00E94D50286E00D
:100F900063EE0E94D50287E06EEA0E94D50285E0EA
:100FA00060E00E94D50286E064EE0E94D50287E0F0
:100FB0006FEA0E94D50285E060E00E94D50286E0DB
:100FC0006BEF0E94D50287E060EB0E94D50285E0BE
:100FD00060E00E94D50286E06CEF0E94D50287E0B7
:100FE00061EB0E94D50285E060E00E94D50286E0B8
:100FF0006DEF0E94D50287E062EB0E94D50285E08A
:1010000060E00E94D50286E06EEF0E94D50287E084
:1010100063EB0E94D50285E060E00E94D50286E085
:101020006FEF0E94D50287E064EB0E94D50285E055
:1010300061E00E94D50286E060E00E94D50287E070
:1010400065EB0E94D50285E061E00E94D50286E052
:1010500061E00E94D50287E066EB0E94D502089508
:10106000BF92CF92DF92EF92FF920F931F93CF9395
:10107000DF937C01B62E8C0145E0C42ED12CC80E26
:10108000D91E862F90E0EC01CC0FDD1FC80FD91FB1
:10109000C25EDE4F0EC085E0612F0E94D50286E061
:1010A000602F0E94D50287E068810E94D5020F5F01
:1010B0001F4F0C151D0578F38701065F1F4F8FE04A
:1010C00090E0E80EF91E8B2D90E0EC01CC0FDD1FB7
:1010D000C80FD91FC25EDE4F0EC085E0612F0E948F
:1010E000D50286E0602F0E94D50287E068810E94C9
:1010F000D5020F5F1F4F0E151F0578F3DF91CF91BB
:101100001F910F91FF90EF90DF90CF90BF900895C7
:10111000EF92FF920F931F93CF93DF938C01EC011B
:1011200055E0E52EF12CE80EF91E0DC085E06D2F7F
:101130000E94D50286E06C2F0E94D50287E060E015
:101140000E94D5022196CE15DF0580F3E8012A968C
:10115000015F1F4F0DC085E06D2F0E94D50286E014
:101160006C2F0E94D50287E060E00E94D502219694
:10117000C017D10780F3DF91CF911F910F91FF909E
:10118000EF9008951F93CF93DF93C0916502D091A4
:101190006602D7FD12C0CE016AE070E00E94851C95
:1011A000182F169520910C0130E0CE016AE070E016
:1011B0000E94851C261B310918C0EE27FF27EC1B57
:1011C000FD0BCF016AE070E00E94851C182F169578
:1011D0001C5F20910C0130E02F5F3F4FCF016AE090
:1011E00070E00E94851C260F311DE90175E0CC0FCF
:1011F000DD1F7A95E1F7220F331FC21BD30B279611
:1012000080911A0190911B01C817D90739F080917C
:101210001A0190911B010E94880804C08091E70187
:10122000811721F0CE01612F0E9430081093E70151
:10123000D0931B01C0931A01DF91CF911F910895A4
:10124000CF92DF92EF92FF920F931F93CF93DF9392
:101250008C01E62E85E0612F0E94D50286E0602F8A
:101260000E94D502CE2CDD248CE391E0C80ED91E5D
:1012700087E0F60160810E94D502EEE1EE2EF12CAE
:10128000E00EF11E85E06F2D0E94D50286E06E2DE6
:101290000E94D50287E0F60160810E94D502E80134
:1012A000CC54DF4F025F1E4F85E06D2F0E94D502A8
:1012B00086E06C2F0E94D50287E0F60160810E94D3
:1012C000D5026E96C017D10779F7DF91CF911F91A4
:1012D0000F91FF90EF90DF90CF900895EF92FF92E3
:1012E0000F931F93CF93DF937C0185E06F2D0E94B6
:1012F000D50286E06E2D0E94D50287E060E00E9454
:10130000D5028701025E1F4F85E0612F0E94D50242
:1013100086E0602F0E94D50287E060E00E94D5023F
:10132000E701CC54DF4F8701025F1E4F85E06D2F30
:101330000E94D50286E06C2F0E94D50287E060E013
:101340000E94D5026E96C017D10781F7DF91CF9129
:101350001F910F91FF90EF9008951F93CF93DF930C
:10136000E0916302F0916402F7FD14C0CF016AE0DE
:1013700070E00E94851C182F16951C5F80910D014E
:10138000C82FD0E0CF016AE070E00E94851CC61B28
:10139000D10917C0222733272E1B3F0BC9016AE052
:1013A00070E00E94851C182F169580910D01C82FA2
:1013B000D0E02196C9016AE070E00E94851CC60F4A
:1013C000D11D80911C0190911D01C817D90739F0DA
:1013D00080911C0190911D010E946E0904C08091B2
:1013E000E801811721F0CE01612F0E94200910939E
:1013F000E801D0931D01C0931C01DF91CF911F9193
:10140000089585E060E00E94D50286E06FEC0E94BE
:10141000D50287E06CE80E94D50285E061E00E9479
:10142000D50286E06BE00E94D50287E06DE80E945D
:10143000D5020895EF92FF920F931F93CF93DF93FE
:101440007A019EE1699FB0011124680F711D8B0123
:10145000020F111D10920904EB0115C085E06D2FDC
:101460000E94D50286E06C2F0E94D502809109046B
:10147000F701E80FF11D60818F5F8093090487E019
:101480000E94D5022196C017D10740F3DF91CF917A
:101490001F910F91FF90EF90089560910B0181E0F3
:1014A00045E151E025E00E941A0A0895DF93CF93A9
:1014B00000D000D0CDB7DEB7F89430916B027894AD
:1014C000832F6AE00E94581C282F0E94581C482F26
:1014D000822F0E94581C292F832F0E94581C992369
:1014E00019F48AE08C8301C09C83222319F48AE0DA
:1014F0008A8301C02A83498385E48B8383E061E08A
:10150000AE014F5F5F4F24E00E941A0A0F900F90C8
:101510000F900F90CF91DF910895DF93CF9300D07C
:1015200000D0CDB7DEB780E289839BE09A8381E368
:101530008B839C8381E061E0AE014F5F5F4F21E0D0
:101540000E941A0A8091B901813079F462E0AE01FB
:101550004E5F5F4F21E00E941A0A81E063E0AE0116
:101560004D5F5F4F22E00E941A0A0F900F900F907C
:101570000F90CF91DF910895DF93CF9300D000D0EB
:101580000F92CDB7DEB7DE011196E9E4F1E085E018
:1015900001900D928150E1F760910C018CE0AE0159
:1015A0004F5F5F4F25E00E941A0A0F900F900F9037
:1015B0000F900F90CF91DF91089580E06CE40E942E
:1015C000D50208958091750390917603843B91052F
:1015D00054F08091F70390E02091730330917403ED
:1015E0008217930744F08091E901882371F481E028
:1015F0008093E90108958091E901181624F480E0B0
:101600006CE40E94D5021092E901089580E062E442
:101610000E94D50208958F929F92AF92BF92CF926F
:10162000DF92EF92FF920F931F93DF93CF93CDB78B
:10163000DEB72F970FB6F894DEBF0FBECDBFFE0109
:101640003B9685E0DF011D928A95E9F7809167025C
:10165000909168026EE170E00E94851CCB010197B9
:1016600097FF02C080E090E08E010F5F1F4FB8012E
:101670004AE050E00E941F1CF80101900020E9F7A9
:101680003197FE2EF01A80E0CF2CDD24C7FCD094D9
:10169000F6E08F2E912C8C0E9D1E58010BC0F5018B
:1016A000E00FF11F80810E943A06080D191DF80114
:1016B00080838E2D082F10E0E82EE3940C151D0575
:1016C00074F38093090485E169E0AE01455F5F4FE3
:1016D00025E00E941A0A89E18F1969E0A4012F2DE3
:1016E0000E941A0A2F960FB6F894DEBF0FBECDBF28
:1016F000CF91DF911F910F91FF90EF90DF90CF90EE
:10170000BF90AF909F908F9008958F929F92AF92CD
:10171000BF92CF92DF92EF92FF920F931F93DF93CE
:10172000CF93CDB7DEB72E970FB6F894DEBF0FBEBE
:10173000CDBF19821A821B821C828091CE019091AA
:10174000CF018E010B5F1F4FB8014AE050E00E94AD
:101750001F1CF80101900020E9F73197FE2EF01AC6
:1017600080E0CF2CDD24C7FCD094AAE08A2E912CF7
:101770008C0E9D1E58010BC0F501E00FF11F8081FA
:101780000E943A06080D191DF80180838E2D082F3E
:1017900010E0E82EE3940C151D0574F38093090402
:1017A00085E166E0AE014F5F5F4F24E00E941A0AB8
:1017B00089E18F1966E0A4012F2D0E941A0A8091F9
:1017C000CE019091CF011816190664F485E060E00F
:1017D0000E94D50286E062EC0E94D50287E06CE8A8
:1017E0000E94D5028091CE019091CF0197FF0CC04D
:1017F00085E060E00E94D50286E062EC0E94D5029E
:1018000087E06DE80E94D5028091CE019091CF01D2
:10181000892B61F485E060E00E94D50286E062ECED
:101820000E94D50287E060E00E94D5022E960FB696
:10183000F894DEBF0FBECDBFCF91DF911F910F9106
:10184000FF90EF90DF90CF90BF90AF909F908F90E0
:1018500008958F929F92AF92BF92CF92DF92EF92B4
:10186000FF920F931F93DF93CF93CDB7DEB72B97E4
:101870000FB6F894DEBF0FBECDBFDE011196E6E4D1
:10188000F1E083E001900D928150E1F78E010C5F51
:101890001F4F8091710390917203B8014AE050E0AC
:1018A0000E941F1CF80101900020E9F73197FE2EDD
:1018B000F01A80E0CF2CDD24C7FCD094B8E08B2E4A
:1018C000912C8C0E9D1E58010BC0F501E00FF11FED
:1018D00080810E943A06080D191DF80180838E2D23
:1018E000082F10E0E82EE3940C151D0574F3809387
:1018F00009048DE06EE0AE014F5F5F4F23E00E9470
:101900001A0A80E18F196EE0A4012F2D0E941A0A95
:101910002B960FB6F894DEBF0FBECDBFCF91DF91EF
:101920001F910F91FF90EF90DF90CF90BF90AF90FD
:101930009F908F9008958F929F92AF92BF92DF9267
:10194000EF92FF920F931F93DF93CF93CDB7DEB744
:1019500028970FB6F894DEBF0FBECDBF19828AE07C
:101960008A838091C0019091C1018E010D5F1F4F4C
:10197000B8014AE050E00E941F1CF80101900020CD
:10198000E9F73197E01B80E0EE2EFF24E7FCF094AE
:10199000480106E0A02EB12CAC0EBD1E0BC0F40118
:1019A000E00FF11F80810E943A060A0D1B1DF8010D
:1019B00080838D2D082F10E0D82ED3940E151F058F
:1019C00074F3809309048091C0019091C1018E014C
:1019D0000A5F1F4F0A977CF460910B0181E0AE0112
:1019E0004F5F5F4F21E00E941A0A60910B0182E075
:1019F000A80121E005C060910B0181E0A80122E06F
:101A00000E941A0A8091C2019091C3018E010D5F5C
:101A10001F4FB8014AE050E00E941F1CF8010190DE
:101A20000020E9F73197E01B80E0EE2EFF24E7FC71
:101A3000F094480116E0A12EB12CAC0EBD1E0BC0D7
:101A4000F401E00FF11F80810E943A060A0D1B1D70
:101A5000F80180838D2D082F10E0D82ED3940E1519
:101A60001F0574F3809309048091C2019091C30112
:101A70008E010A5F1F4F0A977CF460910B0184E08E
:101A8000AE014E5F5F4F21E00E941A0A60910B0188
:101A900085E0A80121E005C060910B0184E0A80168
:101AA00022E00E941A0A28960FB6F894DEBF0FBEF5
:101AB000CDBFCF91DF911F910F91FF90EF90DF90FD
:101AC000BF90AF909F908F9008950F931F93DF93D7
:101AD000CF93CDB7DEB72A970FB6F894DEBF0FBE0F
:101AE000CDBF8E010F5F1F4FB8014AE050E00E944A
:101AF0001F1CF80101900020E9F73197E01B20E05E
:101B0000FF27E7FDF095322F3F5F822F90E08E1781
:101B10009F0714F4232FF7CF209309042A960FB6BA
:101B2000F894DEBF0FBECDBFCF91DF911F910F9113
:101B30000895AF92BF92CF92DF92EF92FF920F93F0
:101B40001F93DF93CF93CDB7DEB76E970FB6F894A0
:101B5000DEBF0FBECDBFB82EA62ED42EA42FB52F1C
:101B6000FD0101900020E9F73197CE2EC41A7E01C5
:101B70000894E11CF11C242F352FC9018C0108C0E9
:101B8000F80181918F010E943A06F70181937F014C
:101B9000802F8D198C15A0F38B2D6A2DAE014F5F10
:101BA0005F4F2C2D0E941A0A6E960FB6F894DEBF76
:101BB0000FBECDBFCF91DF911F910F91FF90EF909E
:101BC000DF90CF90BF90AF9008958091B8018130A1
:101BD00071F460910E012091FF0130910002369561
:101BE00027958EE0821B41E052E00E94990D0895F6
:101BF000EF92FF920F931F93DF93CF93CDB7DEB792
:101C000064970FB6F894DEBF0FBECDBFF82EE62E58
:101C1000CA018E010F5F1F4FB8014AE050E00E94D9
:101C20001F1C8F2D6E2DA8010E94990D64960FB672
:101C3000F894DEBF0FBECDBFCF91DF911F910F9102
:101C4000FF90EF900895EF92FF920F931F93DF9311
:101C5000CF93CDB7DEB72A970FB6F894DEBF0FBE8D
:101C6000CDBF2091B003822F6AE00E94641C382F00
:101C7000822F6AE00E94641C85E48F838091B10307
:101C8000882309F48AE08887992319F48AE08E83EF
:101C900001C09E833D8319821A821B821C8283E0CD
:101CA00062E0AE014B5F5F4F24E00E941A0A809110
:101CB000B4039091B5038952934234F088E293E2E1
:101CC0009093B5038093B4038091B4039091B503CE
:101CD00097FF04C01092B5031092B4038E010B5FFE
:101CE0001F4F8091B4039091B503B8014AE050E0D2
:101CF0000E941F1CF80101900020E9F77F01089461
:101D0000E108F108E01AF10A83E063E0AE014F5FF9
:101D10005F4F24E00E941A0A87E08E1963E0A80151
:101D20000E94990D2A960FB6F894DEBF0FBECDBF64
:101D3000CF91DF911F910F91FF90EF900895BF9287
:101D4000CF92DF92EF92FF920F931F93DF93CF9387
:101D5000CDB7DEB764970FB6F894DEBF0FBECDBF28
:101D6000C82EB62EFA017E010894E11CF11C04C0B5
:101D7000AE0DBF1D9C9331968E2F841B9491A82F7E
:101D8000B0E09923A9F7AE0DBF1D1C92F701019099
:101D90000020E9F73197DE2EDE18870107C0F80131
:101DA00080810E943A06F80181938F01802F8E195D
:101DB0008D15A8F38C2D6B2DAE014F5F5F4F2D2D30
:101DC0000E941A0A64960FB6F894DEBF0FBECDBF0C
:101DD000CF91DF911F910F91FF90EF90DF90CF9007
:101DE000BF9008951F93CF93DF93EC01A3E0B0E081
:101DF00047C0FD01E956FD4F8081FD01E856FD4FCA
:101E00002081422F50E04D535040FD01E756FD4FD9
:101E10007081FD01E656FD4F10819A01F4E0359581
:101E20002795FA95E1F790E0CD97880F991F880FD5
:101E3000991F282B392B2883613029F1E72FF0E0F7
:101E4000FD9734E0440F551F3A95E1F75070CF01EC
:101E50009595879595958795482B592B49836230A1
:101E600091F01496635086E0EE0FFF1F8A95E1F71C
:101E7000F070812F90E0CD97E82BF92BEA83239621
:101E8000662309F0B6CFDF91CF911F9108951F937C
:101E90001091DA01123009F479C0143009F4CEC07F
:101EA000113009F08EC1809199028135A9F48EE438
:101EB00091E06CE00E942E128DED93E062E343E02E
:101EC0002DE20E94F20E8091DD0390E09093DD01FF
:101ED0008093DC011093E00180919902843409F031
:101EE00070C18FE593E061E443E021E40E94F20ECB
:101EF0008091750390917603843B91053CF4809129
:101F0000BA01813051F41092BA0107C08091BA0130
:101F1000882319F481E08093BA0180916103909144
:101F2000620365EF7FEF0E94851C6E5F7F4F7093A9
:101F300066026093650280916303909164036BE095
:101F400070E00E94851C6A5F7F4F7093640260930B
:101F5000630280916B0390916C039093680280936D
:101F600067028091730380936B0280914A02909183
:101F70004B0290936A028093690280917103909161
:101F8000720390936E0280936D021BC1809199023F
:101F90008F34A9F0813509F014C18DED93E062E32F
:101FA00043E02DE20E94F20E8091DD0390E09093D9
:101FB000DD018093DC0181E08093E00102C185E1D5
:101FC00092E060E543E02DE20E94F20E809155021E
:101FD000992787FD909502969093660280936502FB
:101FE00080915602992787FD9095069690936402FA
:101FF0008093630280914802909149029093680215
:102000008093670280914E0280936B0280914A0216
:1020100090914B0290936A028093690280915302DF
:102020009091540290936E0280936D0280914702CA
:1020300080936F0281E08093DF01C3C08091990299
:10204000843409F05AC08FE593E061E443E021E471
:102050000E94F20E8091750390917603843B910566
:1020600054F48091BA01813031F41092BA01F8949D
:102070000E941C1178948091750390917603843BA3
:1020800091057CF08091BA01882359F481E0809316
:10209000BA01F8948091B701882311F40E940C11C1
:1020A0007894809161039091620366E170E00E94F0
:1020B000851C6E5F7F4F709366026093650280910E
:1020C00063039091640366E170E00E94851C6A5F7F
:1020D0007F4F709364026093630280916B039091D1
:1020E0006C039093680280936702809171039091D2
:1020F000720390936E0280936D02809199028C34EA
:1021000081F481E090E09093DD018093DC0181E037
:102110008093E0018FED93E069E143E02DE20E94BE
:10212000F20E809199028D3481F482E090E09093D8
:10213000DD018093DC0181E08093E0018FED93E08D
:1021400069E143E02DE20E94F20E809199028E3403
:1021500081F483E090E09093DD018093DC0181E0E5
:102160008093E0018FED93E069E143E02DE20E946E
:10217000F20E809199028F3481F484E090E0909384
:10218000DD018093DC0181E08093E0018FED93E03D
:1021900069E143E02DE20E94F20E809199028035C0
:1021A00081F485E090E09093DD018093DC0181E093
:1021B0008093E0018FED93E069E143E02DE20E941E
:1021C000F20E1092B5011F91089580919902863503
:1021D00001F58091980281568093DA018091DA01AD
:1021E000843018F084E08093DA018BE591E069E0B7
:1021F0000E942E128091DA01805D0E942A1281EAEB
:1022000093E06AE043E02AE00E94F20E81E08093CE
:10221000DB011092B501089582E289B910BC80B942
:102220001CBE909A28E92AB996E890BD82EC8BB939
:1022300021B99CBF82B9089582E289B910BC80B9E6
:102240001CBE88E98AB926E820BD92EC9BB980E9DA
:1022500081B92CBF92B90895DF93CF93CDB7DEB784
:102260002C970FB6F894DEBF0FBECDBF83E28983F3
:1022700083E68A8385E78B838DE38C838D838E83CE
:102280008F83DE011196FD0120E030E0AE01485F52
:102290005F4F8191280F311DE417F507D1F7C90170
:1022A0009F7046E0959587954A95E1F7835C88870E
:1022B0002F733070822F835C89878DE08A879E011F
:1022C000255F3F4F8C91159BFECF83B91196A217C6
:1022D000B307C1F72C960FB6F894DEBF0FBECDBF83
:1022E000CF91DF910895DF93CF93CDB7DEB72C97D1
:1022F0000FB6F894DEBF0FBECDBF8BE189838A8312
:1023000085E58B838AEA8C831D82FE0131969E01CE
:102310002A5F3F4F8081159BFECF83B93196E2172C
:10232000F307C1F72C960FB6F894DEBF0FBECDBFF2
:10233000CF91DF910895DF93CF93CDB7DEB72A9782
:102340000FB6F894DEBF0FBECDBF93E299838A83A8
:102350006B83842F86958695835C8C8350E04370D5
:10236000507064E0440F551F6A95E1F7435C4D835C
:102370008DE38E838F83DE011196FD0120E030E036
:10238000AE01485F5F4F8191280F311DE417F507BB
:10239000D1F7C9019F7056E0959587955A95E1F759
:1023A000835C88872F733070822F835C89878DE0F0
:1023B0008A879E01255F3F4F8C91159BFECF83B985
:1023C0001196A217B307C1F72A960FB6F894DEBF8D
:1023D0000FBECDBFCF91DF9108955D9BFECF8DE6FF
:1023E0008CB95D9BFECF8FE68CB95D9BFECF89E6F5
:1023F0008CB95D9BFECF8EE68CB95D9BFECF8DE0E8
:102400008CB95D9BFECF8EE38CB90895982F9F7099
:1024100082958F708A3010F4805D01C0895C5D9B6D
:10242000FECF8CB99A3018F4892F805D02C0892FB5
:10243000895C5D9BFECF8CB908958A3010F4805D75
:1024400001C0895C5D9BFECF8CB90895159BFECFC2
:1024500083B908955D9BFECF8CB90895662359F02A
:1024600020E0FC01E20FF11DE0815D9BFECFECB9A5
:102470002F5F6217B0F708955D9BFECF8EE38CB996
:1024800008951F920F920FB60F9211242F933F932E
:102490008F939F93AF93BF93EF93FF932CB12093B0
:1024A0000A0485B398E0892785BB5D9BFECF2CB9D4
:1024B0002D3059F08091DC03E82FF0E0EA54FC4F16
:1024C00020838F5F8093DC035FC0E091DC03F0E04A
:1024D000EA54FC4F20831092D7011092D801109239
:1024E000D90130E020E090E045C02130B9F0213042
:1024F00018F02230F1F528C0A32FB0E0AA54BC4F49
:102500008C91803211F421E033C0E92FF0E08C91FE
:10251000EC52FC4F80839093D7010FC0A32FB0E003
:10252000AA54BC4F8C91E92FF0E0803241F08C919D
:10253000E657FD4F80839093D8019F5F1AC0E657FE
:10254000FD4F108222E014C0A32FB0E0AA54BC4F6C
:102550008C91E92FF0E08D3039F08C91EF58FD4FE0
:1025600080839093D901E9CFEF58FD4F108223E08B
:1025700090E03F5F8091DC03831708F0B6CF81E0E5
:102580008093D6011092DC03FF91EF91BF91AF9140
:102590009F918F913F912F910F900FBE0F901F90A1
:1025A00018951F920F920FB60F9211248F939F933D
:1025B000EF93FF9393B190930B049CB99D3081F4FA
:1025C0008091EA01813061F4AB981092EA01809326
:1025D000B501E091AC03F0E0E956FD4F90832DC0CA
:1025E0008091EA01882319F0813039F514C09332C3
:1025F00041F48091B501882321F481E08093EA01C0
:10260000AB9A1092AC038091AC03E82FF0E0E9564E
:10261000FD4F90830CC0E091AC03F0E0E956FD4F14
:1026200090838091AC03873C30F48091AC038F5F42
:102630008093AC0302C01092EA01FF91EF919F9149
:102640008F910F900FBE0F901F90189585B392E059
:10265000892785BB08959091BD01913019F485B308
:10266000892785BB08951F920F920FB60F921124F0
:102670002F933F935F936F937F938F939F93AF932A
:10268000BF938091EC019091ED01892B81F484B589
:1026900095B59093F3018093F2018EB58F7B8EBD3B
:1026A00081E090E09093ED018093EC013AC084B515
:1026B00095B59093F1018093F0012EB520642EBD65
:1026C0002091F2013091F3011092ED011092EC0192
:1026D000821B930B865698406CE271E00E94711C3D
:1026E0007093EF016093EE016730710534F086E07E
:1026F00090E09093EF018093EE012091EE013091F4
:10270000EF0180910A01992787FD909528173907D5
:1027100041F0263031052CF420930A0181E08093AA
:10272000C401BF91AF919F918F917F916F915F9104
:102730003F912F910F900FBE0F901F901895809191
:102740006702909168029093C7018093C6018091BF
:10275000C6019091C7012091C8013091C901821B27
:10276000930B9093CB018093CA018091C601909105
:10277000C7019093C9018093C8014091D201509143
:10278000D3018091CA019091CB01E3E0880F991F9A
:10279000EA95E1F79A0173E0220F331F7A95E1F78A
:1027A000241B350B820F931F68E070E00E94851C8C
:1027B0007093D3016093D2012091D4013091D5015F
:1027C0004091D2015091D301C90163E0880F991F54
:1027D0006A95E1F7821B930B840F951F68E070E008
:1027E0000E94851C7093D5016093D4018091D4011F
:1027F0009091D5019093CF018093CE010E94850BDB
:10280000089560910C018BE14DE651E00E94990D15
:102810008091590281FF07C060910C018BE140E774
:1028200051E00E94990D8091590282FF07C060918A
:102830000C018BE143E751E00E94990D0895DF936D
:10284000CF930F92CDB7DEB78091430290914402AF
:1028500021E0823592071CF080EC898307C04E96F8
:102860006DE270E00E94851C6054698360910C01E8
:102870008EE0AE014F5F5F4F21E00E941A0A0F9079
:10288000CF91DF9108958AE161E046E751E022E0CF
:102890000E941A0A0895DF93CF9300D000D0CDB7DD
:1028A000DEB719821A821B821C8260910B01615073
:1028B00085E1AE014F5F5F4F24E00E941A0A6091EC
:1028C0000B016150409130025091310285E10E942C
:1028D000F80D0F900F900F900F90CF91DF9108950A
:1028E000DF93CF9300D00F92CDB7DEB7DE01119604
:1028F000E8E7F1E083E001900D928150E1F760910B
:102900000C016F5F8EE0AE014F5F5F4F23E00E94CE
:102910001A0A20910C012F5F80914102909142028E
:102920006AE070E00E94851CAB018EE0622F0E947D
:10293000F80D0F900F900F90CF91DF9108958F9227
:102940009F92BF92CF92DF92EF92FF920F931F93CD
:10295000DF93CF93CDB7DEB72B970FB6F894DEBFDA
:102960000FBECDBFDE011196EBE7F1E083E00190F1
:102970000D928150E1F780916F028E010C5F1F4F25
:1029800090E0B8014AE050E00E941F1CF80101905D
:102990000020E9F73197BE2EB01AEE24FF24CB2C8D
:1029A000DD24C7FCD09488E0882E912C8C0E9D1ECF
:1029B0000DC0F801EE0DFF1D80810E943A06F40162
:1029C000EE0DFF1D80830894E11CF11CEC14FD0446
:1029D00084F388E161E0AE014F5F5F4F23E00E9426
:1029E0001A0A8BE18B1961E0A4012B2D0E941A0AAF
:1029F0002B960FB6F894DEBF0FBECDBFCF91DF91FF
:102A00001F910F91FF90EF90DF90CF90BF909F901C
:102A10008F9008958F929F92BF92CF92DF92EF9204
:102A2000FF920F931F93DF93CF93CDB7DEB76A97D3
:102A30000FB6F894DEBF0FBECDBFFE01319686E023
:102A4000DF011D928A95E9F720914F0230915002E3
:102A5000C90143E0880F991F4A95E1F7820F931F40
:102A60006AEF70E00E94711CCB018E01095F1F4F5D
:102A7000B8014AE050E00E941F1CF80101900020BC
:102A8000E9F73197BE2EB01AEE24FF24CB2CDD24BB
:102A9000C7FCD09491E1892E912C8C0E9D1E0DC007
:102AA000F801EE0DFF1D80810E943A06F401EE0D43
:102AB000FF1D80830894E11CF11CEC14FD0484F3D9
:102AC00060910B0185E1AE014F5F5F4F26E00E94F0
:102AD0001A0A60910B018BE18B19A4012B2D0E9426
:102AE0001A0A6A960FB6F894DEBF0FBECDBFCF911B
:102AF000DF911F910F91FF90EF90DF90CF90BF90EB
:102B00009F908F90089583E66FE644E60E949B11A4
:102B1000F89428E088E190E00FB6F894A89581BD7C
:102B20000FBE21BDFFCF1F939D998AC18091F401F3
:102B30008F5F8093F40111E01093F6018091F4010E
:102B4000853009F081C18091F801882309F08CC09B
:102B50001093F8011092F90184E064E00E94D5021C
:102B600083E061E041E052E00E94990D83E063E080
:102B700040E152E00E949F0E84E068E00E94D5028E
:102B800083E065E049E152E00E949F0E80910801D8
:102B9000813029F484E165E045E452E004C084E139
:102BA00065E048E452E00E949F0E84E060E00E94ED
:102BB000D50283E066E04DE152E00E949F0E8091D5
:102BC000B701813029F484E166E045E452E004C0B5
:102BD00084E166E048E452E00E949F0E83E067E0F3
:102BE00043E252E00E949F0E8091B801813029F4A7
:102BF00084E167E045E452E004C084E167E048E432
:102C000052E00E949F0E83E068E04BE252E00E9497
:102C10009F0E8091C501813029F484E168E045E48C
:102C200052E004C084E168E048E452E00E949F0E54
:102C300083E069E046E352E00E949F0E8091B90173
:102C4000813029F484E169E045E452E004C084E184
:102C500069E048E452E00E949F0E83E06BE040E4AC
:102C600052E00E949F0EEEC08091F901882349F541
:102C700084E068E00E94D50280910801882339F43D
:102C80001093080184E165E045E452E006C010922B
:102C9000080184E165E048E452E00E949F0E209123
:102CA0000801E199FECF81E090E09FBB8EBB2DBB78
:102CB0000FB6F894E29AE19A0FBE84E060E00E94B9
:102CC000D5021091F901113049F584E068E00E94C5
:102CD000D5028091B701882339F41093B70184E1BC
:102CE00066E045E452E006C01092B70184E166E078
:102CF00048E452E00E949F0E2091B701E199FECF77
:102D000080E090E09FBB8EBB2DBB0FB6F894E29A9B
:102D1000E19A0FBE84E060E00E94D5028091F90143
:102D2000823051F584E068E00E94D5028091B801BC
:102D3000882341F481E08093B80184E167E045E4B1
:102D400052E006C01092B80184E167E048E452E026
:102D50000E949F0E2091B801E199FECF82E090E0A1
:102D60009FBB8EBB2DBB0FB6F894E29AE19A0FBEC3
:102D700084E060E00E94D5028091F901833051F532
:102D800084E068E00E94D5028091C501882341F467
:102D900081E08093C50184E168E045E452E006C02B
:102DA0001092C50184E168E048E452E00E949F0E61
:102DB0002091C501E199FECF87E190E09FBB8EBBDA
:102DC0002DBB0FB6F894E29AE19A0FBE84E060E062
:102DD0000E94D5028091F901843049F568E00E9493
:102DE000D5028091B901882341F481E08093B90133
:102DF00084E169E045E452E006C01092B90184E143
:102E000069E048E452E00E949F0E2091B901E199E7
:102E1000FECF8BE190E09FBB8EBB2DBB0FB6F8942D
:102E2000E29AE19A0FBE84E060E00E94D5028091B0
:102E3000F901853049F41092F8010E94831504C00D
:102E40001092F4011092F6019C9913C19091F8012F
:102E5000913009F014C19093F7018091F5018F5FD3
:102E60008093F5012091F501253009F008C11092F9
:102E7000F5018091F901823009F469C0833030F4A2
:102E8000882371F0813009F0FAC035C0843009F42C
:102E9000AAC0843008F486C0853009F0F0C0C3C0F1
:102EA0009093F90183E065E049E152E00E949F0EB2
:102EB00080910801813029F484E165E045E452E025
:102EC00004C084E165E048E452E00E949F0E84E083
:102ED00068E00E94D50283E066E04DE152E00E9486
:102EE0009F0E8091B701813019F484E166E0B3C090
:102EF00084E166E0B5C082E08093F90183E066E09A
:102F00004DE152E00E949F0E8091B701813029F47B
:102F100084E166E045E452E004C084E166E048E410
:102F200052E00E949F0E84E068E00E94D50283E098
:102F300067E043E252E00E949F0E8091B801813029
:102F400019F484E167E087C084E167E089C083E029
:102F50008093F90167E043E252E00E949F0E809166
:102F6000B801813029F484E167E045E452E004C00F
:102F700084E167E048E452E00E949F0E84E068E04C
:102F80000E94D50283E068E04BE252E00E949F0E6F
:102F90008091C501813019F484E168E05CC084E16E
:102FA00068E05EC084E08093F90183E068E04BE272
:102FB00052E00E949F0E8091C501813029F484E186
:102FC00068E045E452E004C084E168E048E452E08F
:102FD0000E949F0E84E068E00E94D50283E069E0D1
:102FE00046E352E03FC02093F90183E069E046E305
:102FF00052E00E949F0E8091B901813029F484E152
:1030000069E045E452E004C084E169E048E452E04C
:103010000E949F0E84E068E00E94D50283E06BE08E
:1030200040E452E01FC01092F90183E06BE040E4FD
:1030300052E00E949F0E84E068E00E94D50283E087
:1030400065E049E152E00E949F0E809108018130C5
:1030500029F484E165E045E452E004C084E165E0E0
:1030600048E452E00E949F0E84E060E00E94D50296
:1030700006C01092F5018091F6018091F7011F9131
:103080000895813061F4E199FECF80E090E09FBB2C
:103090008EBB6DBB0FB6F894E29AE19A0FBE08950D
:1030A000DF93CF93CDB7DEB764970FB6F894DEBF4A
:1030B0000FBECDBF20E0DE011196E199FECFE22FD9
:1030C000F0E0CF018D5F9F4F9FBB8EBBE09A8DB329
:1030D000EA0FFB1F8083882311F02F5FEECFFD01E5
:1030E00001900020E9F79F01215030402A1B3B0B43
:1030F000309300022093FF0190E0AE014F5F5F4FDD
:1031000009C0FD01EF5FFD4FA40FB51F8C918083B7
:1031100011829F5FA92FB0E0A217B30790F36496C6
:103120000FB6F894DEBF0FBECDBFCF91DF910895EB
:10313000DF93CF93CDB7DEB760970FB6F894DEBFBD
:103140000FBECDBF80916D0290916E02909396025A
:103150008093950280919502909196026FE070E0C5
:103160000E94711CDE011596AD016A1B9E01205F55
:103170003F4FE62FEA0FF0E0E55BFD4FE491ED9362
:10318000A217B307B1F760910F0119821A821B824F
:103190001C8289E02BE00E941A0A609110018EE0E7
:1031A000AE014F5F5F4F24E00E941A0A6091100148
:1031B00040919502509196028FE00E94F80D609622
:1031C0000FB6F894DEBF0FBECDBFCF91DF9108954B
:1031D000FF920F931F93DF93CF93CDB7DEB7E397A3
:1031E0000FB6F894DEBF0FBECDBFDE011C96EEE732
:1031F000F1E087E001900D928150E1F7DE015396F6
:10320000E5E8F1E089E001900D928150E1F7DE01FF
:103210009696EEE8F1E08EE001900D928150E1F794
:10322000DE011696ECE9F1E086E001900D92815006
:10323000E1F7DE015C96E2EAF1E08AE001900D92AE
:103240008150E1F78091D4039091D503873409F040
:1032500066C0943409F063C080918A0290918B0219
:10326000813409F05CC09C3409F059C0E199FECF6B
:1032700081E090E09FBB8EBBE09A2DB3211121E04D
:10328000022FE199FECF80E090E09FBB8EBBE09AD9
:103290008DB3882311F0022F0260E199FECF82E006
:1032A00090E09FBB8EBBE09A8DB381110460E199E1
:1032B000FECF87E190E09FBB8EBBE09A8DB381117A
:1032C0000860E199FECF8BE190E09FBB8EBBE09A56
:1032D0008DB38111006183E20E942A12802F90E059
:1032E0008E010F5F1F4FB8014AE050E00E941F1C83
:1032F000F80101900020E9F73197E01BF10BC801BC
:103300006E2F0E942E128CE20E942A1281E092E01F
:103310006091FF010E942E128DE00E942A1280917E
:10332000D4039091D503833509F0B6C0943409F0E5
:10333000B3C08AE892E00E94FA1BF82E01E012E086
:10334000C80161E772E00E94181CD8010D900020AE
:10335000E9F71197A01BB10B80E011C0F901EF5FF5
:10336000FD4FE081E199FECF2D5F3F4F3FBB2EBB6C
:10337000EDBB0FB6F894E29AE19A0FBE8F5F282F4B
:1033800030E02A173B0750F3E199FECF8F5F90E0C2
:103390008D5F9F4F9FBB8EBB1DBA0FB6F894E29A0C
:1033A000E19A0FBEB0930002A093FF012F2DF0FE13
:1033B00009C0E199FECF81E090E09FBB8EBB81E028
:1033C0008DBB07C0E199FECF81E090E09FBB8EBB33
:1033D0001DBA0FB6F894E29AE19A0FBE21FF09C018
:1033E000E199FECF80E090E09FBB8EBB81E08DBB7A
:1033F00007C0E199FECF80E090E09FBB8EBB1DBA75
:103400000FB6F894E29AE19A0FBE22FF09C0E19943
:10341000FECF82E090E09FBB8EBB81E08DBB07C0FA
:10342000E199FECF82E090E09FBB8EBB1DBA0FB644
:10343000F894E29AE19A0FBE23FF09C0E199FECF0A
:1034400087E190E09FBB8EBB81E08DBB07C0E19917
:10345000FECF87E190E09FBB8EBB1DBA0FB6F894FC
:10346000E29AE19A0FBE24FF09C0E199FECF8BE1F9
:1034700090E09FBB8EBB81E08DBB07C0E199FECF82
:103480008BE190E09FBB8EBB1DBA0FB6F894E29A19
:10349000E19A0FBE0E9483155091D4036091D50329
:1034A0004091D6038091D70320E030E0803711F4BB
:1034B00021E030E080E090E04C3611F481E090E0D3
:1034C0002823392380E0583609F481E090E06536FE
:1034D00009F491E0892390E028233923232B79F004
:1034E000CE010C9666E00E942E12CE01439668E053
:1034F0000E942E12CE0186966DE00E942E125091EF
:10350000D4036091D5034091D6038091D70320E086
:1035100030E0873711F421E030E080E090E04F3672
:1035200011F481E090E02823392380E0533709F437
:1035300081E090E0683609F491E0892390E0282347
:103540003923232B19F180918A0290918B028934BF
:1035500081F4943471F4CE01069665E00E942E1237
:1035600081E092E06091FF010E942E128DE00E94A6
:103570002A1280918A0290918B02863739F495360F
:1035800029F4CE014C966CE00E942E128091D40357
:103590002091D5034091D60390E0833709F491E060
:1035A00080E0253609F481E09823892F90E020E01F
:1035B00030E0443711F421E030E082239323892B5B
:1035C00009F442C080918A0290918B02893409F0FB
:1035D0003BC0943409F038C020E01AC0FD01EF5818
:1035E000FD4FE081E199FECF822F90E08D5F9F4FEC
:1035F0009FBB8EBBEDBB0FB6F894E29AE19A0FBE6B
:10360000FD01EF58FD4F8081AF5FBD4F8C932F5F61
:103610008091D901A22FB0E0281700F3E199FECFE5
:10362000CD018D5F9F4F9FBB8EBB1DBA0FB6F89427
:10363000E29AE19A0FBEE22FF0E0EF5FFD4F1082B9
:10364000B0930002A093FF015091D4036091D50381
:103650004091D6038091D70320E030E0853611F405
:1036600021E030E080E090E0433711F481E090E029
:103670002823392380E0523709F481E090E0653651
:1036800009F491E0892390E028233923232B11F0BA
:103690000E948315E3960FB6F894DEBF0FBECDBF30
:1036A000CF91DF911F910F91FF9008951F920F927C
:1036B0000FB60F9211242F933F938F939F93EF9305
:1036C000FF938091FB01882381F08091FB0190E0C2
:1036D0000197E091AE01F091AF01E80FF91F8FB1B2
:1036E000808381E08093FC0103C08FB1809311043B
:1036F0002091FB018091AC0130E0992787FD9095E6
:10370000821793075CF084E08093AD0181E08093A1
:10371000FC018091FB018093100408C0929A1092E2
:10372000FA0181E08093FD011092FE018091FB017E
:103730008F5F8093FB01FF91EF919F918F913F915C
:103740002F910F900FBE0F901F90189582ED8DB99D
:103750000895813029F4613011F492980895929A75
:103760000895982F8091FA018823C9F4913009F4C3
:1037700092989093FA0181E08093FE01913069F470
:1037800086E08093AC011092FB018AE08093AD014A
:103790009093FC018AEA8093100480E00895809160
:1037A000FC01813071F48091AD0181508093AD01B5
:1037B0008F5F39F4809110048FB91092FC0181E081
:1037C000089581E00895CF93DF93C0E0D0E0E091C9
:1037D000AE01F091AF01EC0FFD1F80810E94061237
:1037E0002196C730D10599F78DE00E942A12DF910A
:1037F000CF910895FC0188279927E89421912032E0
:10380000E9F3293010F02E30C8F32B3241F02D327D
:1038100039F4689404C00E94401C820F911D2191CC
:1038200020532A30C0F31EF4909581959F4F089540
:10383000FB01DC0101900D920020E1F70895FB01EE
:103840009F01E8944230C4F04532B4F44A3029F480
:1038500097FB1EF4909581959F4F642F77270E94C8
:10386000711C805D8A330CF0895D8193CB010097D8
:10387000A1F716F45DE251931082C9010C94481C23
:103880007AE0979F902D879F802D910D11240895A8
:10389000DC01FC01672F71917723E1F7329704C0B7
:1038A0007C916D9370836291AE17BF07C8F3089542
:1038B000991B79E004C0991F961708F0961B881F82
:1038C0007A95C9F78095089587FB082E062687FD0F
:1038D000819567FD6195ECDF0EF4919507FC81956C
:1038E0000895AA1BBB1B51E107C0AA1FBB1FA61747
:1038F000B70710F0A61BB70B881F991F5A95A9F799
:1039000080959095BC01CD01089597FB092E07265F
:103910000AD077FD04D0E5DF06D000201AF47095B8
:1039200061957F4F0895F6F7909581959F4F089583
:04393000F894FFCF39
:1039340053656E6420640D000101030E0786010EB9
:103944000C5C00000A0000440000230023005464BF
:10395400665363655262005161005060005060001C
:103964005161005262005363655464666768696A12
:103974006B6B6A69686700000053536353532053A9
:10398400657474696E6720656D700044657669635B
:1039940065203D20005F031502DD030D0A20200091
:1039A4005048004348000A1D0000000000006865FC
:1039B4006C70200D0073686F772049440D007368A4
:1039C4006F772076657273696F6E0D004944203DF0
:1039D4002000302E392E342E302E31000907AF034B
:00000001FF
